:1000000012C0189518951895189518951895189563
:1000100072C01895189518951895189518951895F3
:100020001895189518958FE58DBFC0EEE8E64E2E11
:1000300084E08EBFD3E0F3E05F2EEEEFF3E0A0E6C6
:10004000B0E084B7082E877F84BF8FE181BD80E058
:1000500081BD88278D933197E9F7662480E08FBDB5
:1000600084E08EBDB89AA198A098A59AA49AA39A64
:10007000A29A9D989C989B989A988F9A8E9A8D9AFE
:100080008C9A9798969895989498A99AA89A89B7CF
:10009000846089BF789470D0E4D0F5D0A198A2E6AE
:1000A000B0E09C9197FF04C0999B0EC09F779C93F2
:1000B00099990AC089E19F9399270AD19F919999AB
:1000C00003C090689C939FD0A098A2E6B0E09C915A
:1000D00096FF04C0989B0EC09F7B9C9398990AC082
:1000E00089E19F939927F4D09F91989903C09064D8
:1000F0009C93A0D0D3CF0F921F922F923F924F92FA
:100100005F927F92AF92BF920F931F932F933F9373
:100110004F935F936F937F938F939F93AF93BF930F
:10012000CF93DF93EF93FF938FB78F938EEE95E886
:1001300090934D0080934C0088B391E0892788BB51
:100140008F918FBFFF91EF91DF91CF91BF91AF91D1
:100150009F918F917F916F915F914F913F912F91DF
:100160001F910F91BF90AF907F905F904F903F9005
:100170002F901F900F901895E0E0F0E0A0E6B0E01F
:10018000CDD0E1E0F0E0A1E6B0E0C8D000916000A1
:10019000013008F009C081E080936000E0E0F0E009
:1001A000A0E6B0E07BE7A9D000916000023010F03B
:1001B00009F001C009C082E080936000E0E0F0E057
:1001C000A0E6B0E07BE799D000916100013008F033
:1001D00009C081E080936100E1E0F0E0A1E6B0E0D9
:1001E0007BE78BD000916100033010F009F001C073
:1001F00009C083E080936100E1E0F0E0A1E6B0E0B7
:100200007BE77BD00895A0E6B0E08C918F5F8C9364
:1002100000916000023010F009F001C003C081E0DD
:1002200080936000E0E0F0E0A0E6B0E07BE765D01E
:1002300018D00895A1E6B0E08C918F5F8C93009167
:100240006100033010F009F001C003C081E0809329
:100250006100E1E0F0E0A1E6B0E07BE74ED013D032
:10026000089500916000013009F005C0AC9897989E
:10027000AD9A969A07C0023009F004C0AD989698DE
:10028000AC9A979A089500916100013009F005C079
:10029000AB9A9598AA98949A0FC0023009F005C0BD
:1002A000AB98959AAA9A949807C0033009F004C0B5
:1002B000AB9A9598AA9A94980895F894FFCF31979D
:1002C000F1F70895689462F80895E89462F8089543
:1002D000EF93FF93EE27E82BE92B31F0E0EDF7E009
:1002E0003197F1F70197D1F7FF91EF910895E199D7
:1002F000FECFEEBBFFBB3196089591E001C092E0C6
:100300007B3751F47FB7F894F2DF8D918DBBE29A81
:10031000E19A9A95C9F77FBF7727089591E001C0C8
:1003200092E0E5DFE09A8DB38D939A95D1F7089529
:00000001FF
